:1000000012C02CC02BC02AC029C028C027C026C0BF
:1000100025C024C023C022C021C020C01FC01EC0D4
:100020001DC01CC01BC011241FBECFE5D4E0DEBF25
:10003000CDBF10E0A0E6B0E0EEEBF4E002C005902A
:100040000D92A036B107D9F710E0A0E6B0E001C0EC
:100050001D92A036B107E1F70FD230C2D1CF8099FF
:1000600026C024EF31E080E991E00197F1F72150BB
:100070003040C9F724EF31E080E991E00197F1F7D2
:1000800021503040C9F7809B12C024EF31E080E955
:1000900091E00197F1F721503040C9F724EF31E0AA
:1000A00080E991E00197F1F721503040C9F781993B
:1000B00026C024EF31E080E991E00197F1F721506B
:1000C0003040C9F724EF31E080E991E00197F1F782
:1000D00021503040C9F7819B12C024EF31E080E904
:1000E00091E00197F1F721503040C9F724EF31E05A
:1000F00080E991E00197F1F721503040C9F7089568
:10010000482F24EC39E080E991E00197F1F7215084
:100110003040C9F7842FA3DF24EC39E080E991E077
:100120000197F1F721503040C9F708958CEF82BB59
:1001300087E088BB8FE385BB089582B382BB88B319
:1001400088BB85B385BB0895982F813021F480E268
:1001500085BB98BB0895823009F4A2C0833009F4AE
:10016000A4C0843009F4A6C0853009F4A8C0863044
:1001700009F4AAC0873009F4ACC0883021F4929801
:10018000AD9880E147C0893009F48AC08A3009F40B
:100190008CC08B3009F48EC08C3009F490C08D3047
:1001A00009F492C08E3009F494C08F3021F49298F3
:1001B000AC9888E02FC0803109F472C0813109F415
:1001C00074C0823109F476C0833109F478C0843177
:1001D00009F47AC0853109F47CC0863121F4929803
:1001E000AB9884E017C0873109F45AC0883109F40C
:1001F0005CC0893109F45EC08A3109F460C08B317A
:1002000009F462C08C3109F464C08D3129F49298EC
:10021000AA9882E085BB3FC08E3109F441C08F317E
:1002200009F443C0803219F4969882BB0895813254
:1002300009F445C0823209F447C0833209F449C049
:10024000843229F49298A99881E085BB25C0853233
:1002500039F1863251F1873269F1883281F1893280
:1002600099F18A32B1F18B3221F49298A89884E006
:1002700011C08C32A9F08D32C1F08E32D9F08F329C
:10028000F1F0803309F1813321F1823339F492980E
:10029000C29882E088BB81E088BB0895833319F45B
:1002A000C09880E818C0843319F4979880E413C08C
:1002B000853319F4969880E20EC0863319F4959828
:1002C00080E109C0873319F4949888E004C088332A
:1002D00021F4939884E082BB0895893311F49298B5
:1002E000C1980895813019F482E088BB9EC08230A5
:1002F00009F49FC0833009F4A1C0843009F4A3C07D
:10030000853009F4A5C0863009F4A8C0873009F407
:10031000AAC0883029F4C098C19884E088BB9AC0EC
:10032000893009F486C08A3009F488C08B3009F41A
:100330008AC08C3009F48CC08D3009F48FC08E30A7
:1003400009F491C08F3021F4C098C29881E06CC04C
:10035000803109F46EC0813109F470C0823109F432
:1003600072C0833109F474C0843109F477C08531D7
:1003700009F479C0863121F4C098A89882E054C06D
:10038000873109F456C0883109F458C0893109F41D
:100390005AC08A3109F45CC08B3109F45FC08C31DA
:1003A00009F461C08D3129F4C098A99884E085BB17
:1003B00051C08E31F1F18F3109F440C0803211F417
:1003C000949848C0813209F443C0823209F446C08F
:1003D000833209F448C0843221F4C098AA9888E096
:1003E00023C0853231F1863249F1873261F188329A
:1003F00079F1893299F18A32B1F18B3221F4C098C6
:10040000AB9880E111C08C32A1F08D32B9F08E3200
:10041000D1F08F32E9F0803309F1813321F1823359
:1004200031F4C098AC9880E285BB84E013C083337C
:1004300019F4929888E00EC0843319F4939880E1FF
:1004400009C0853319F4949880E204C0863321F4FE
:10045000959880E482BB0895873319F4969880E8D4
:10046000F9CF883321F4979881E088BB08958933C8
:1004700011F4C098AD9808951F938CEF81BB87E06D
:1004800087BB8FE384BB83E082BB82B382BB88B32C
:1004900088BB85B385BB14E601C011E061E081E053
:1004A000DEDD113039F08CEF82BB87E088BB8FE353
:0E04B00085BBF3CF61E081E0D2DDEFCFFFCF5F
:00000001FF
